:02000000AEC090
:020010009EC38D
:14002400CEC35BB509000000000000000000000000C000C09E
:140038000000000000000000000000000000000000000000B4
:14004C00000000003838383838380000000000000000000050
:1400600000000000000000000000000000000000000000008C
:14007400000000000000000000000000000000000000000078
:14008800000000000000000000000000000000000000000064
:14009C00000000000000000000000000000000000000000050
:1400B00000000000000000000000000000000000000000003C
:1400C400000000000000000000000000000000000000000028
:1400D800000000000000000000000000000000000000000014
:1400EC00000000000000000000000000000000000000000000
:140100000000000000000000000000000000000000000000EB
:140114000000000000000000000000000000000000000000D7
:140128000000000000000000000000000000000000000000C3
:14013C000000000000000000000000000000000000000000AF
:140150000000000000000000000000000000CFE5D4E0CDBFA7
:14016400DEBFC051D0400AEA08830024E8E9F1E011E0E83A71
:14017800F10711F00192FBCF0083E6E2F0E0A0E6B0E011E0FB
:14018C0000E00BBFEE35F10721F0C89531960D92F9CFC3D269
:1401A000FFCFE2D4442755270BC06627772702C06F5F7F4F8C
:1401B4006634E0E07E07D0F34F5F5F4F4017510790F3D5C46E
:1401C800CFD4442755270BC06627772702C06F5F7F4F6E35A2
:1401DC00E6E07E07D0F34F5F5F4F4017510790F3C2C488E97C
:1401F0008AB98BE089B9222420BC86E880BD88E98AB90895ED
:1402040083E08EBD84E68CBD22242DBC84E089BF80E88FBFF4
:140218008FEF87BB0895A8958FE181BD8FE081BD08958DD4DF
:14022C00C22EE02EAE800E2D1C2DC4D4802F817049F001E0BC
:140240001A2DB8D42090A701202A2092A7010AC001E01A2DE9
:14025400AFD4202E20943090A70132203092A7018091A70134
:14026800806C8093A70155C421978FEF84BB222425BA81B3F4
:14027C00806E81BBB89A959A969AC09A979A8A9A9298BA9A66
:14029000C2988B988C98B998BB98BC98BD98939A949AC19AB6
:1402A400C39AC49AC59A04E610E08CDF95989698C29A85E0CB
:1402B800888325E006B3B5DF84E0888324E006B3B0DF83E0B7
:1402CC00888323E006B3ABDF82E0888321E006B3A6DF81E0C0
:1402E000888324E000B3A1DF2224288223E000B39CDF2090F7
:1402F400A70120942092A701219608955D9BFECF0CB90895C5
:14030800AA92BA925801929A04C0F50101915F01F3DFF50160
:14031C0020802220C1F70DE0EDDF0AE0EBDF5D9BFECF02E01F
:1403300010E04ADF9298B990A990089598D3FFD3C22E4427BF
:14034400242E33244F5F80E690E0E22DFF27E80FF91F8BE5C4
:140358008083242E33244F5F80E690E0E22DFF27E80FF91F1D
:14036C0085EB8083E42EFF244F5F80E690E0EE2DFF27E80F19
:14038000F91F85E08083E42EFF244F5F80E690E0EE2DFF27EF
:14039400E80FF91F2090A7012082E42EFF244F5FEE2DFF2728
:1403A800E80FF91F0A840082E42EFF244F5FEE2DFF27E80F07
:1403BC00F91FC082C42EDD244F5FEC2DFF27E80FF91F209034
:1403D00071002082C42EDD244F5FEC2DFF27E80FF91F209067
:1403E40072002082242F00E610E01FD2C02E6C2DC42EDD245D
:1403F8004F5F80E690E0EC2DFF27E80FF91F6083642F77270B
:14040C004F5FE62FFF27E80FF91F8DE08083642F77274F5F95
:1404200080E690E0E62FFF27E80FF91F8AE08083929A01E02E
:1404340010E0C8DEAA240BC05D9BFECF80E690E0EA2DFF27AD
:14044800E80FF91F20802CB8A394A41698F35D9BFECF01E0EB
:14045C0010E0B4DE929862D324960895AA92A02E2224209252
:1404700072002092710095989698979A24BAC09801E010E050
:14048400A1DEC09AC09823B230907200322830927200C09A44
:14049800979801E010E094DE979A979883B3880F880F880F83
:1404AC00880F880F880F807C20907200282A2092720083B3AD
:1404C000869586958F7080937100C09A979AAA2059F0309011
:1404D4006F00381621F430907000321419F0222702EC2ADF83
:1404E8002090710020926F002090720020927000A9900895A4
:1404FC004A93402F87E991E0E42FFF27E80FF91F2080222095
:1405100009F03CC0959896988FEF84BB8CE08417D0F086E09D
:140524008417B8F416E0042F0150DDD2102F01E03FD3209071
:14053800A601202A2092A60125BA87E991E0E42FFF27E80F75
:14054C00F91F84E08083969A19C086E08417B0F016E0042F49
:140560000150C3D2102F01E025D32090A501202A2092A50191
:1405740025BA87E991E0E42FFF27E80FF91F84E08083959AD5
:1405880095989698499108954A93402F80917300813069F4AF
:14059C00042F0F5FADDF4C3040F022242092730000275CDFA5
:1405B000222703ECC3DE499108954A93402F8CE0841790F014
:1405C40086E0841778F416E0042F01508CD2102F01E0EED2FE
:1405D800202E20943090A60132203092A60111C086E0841719
:1405EC0070F016E0042F01507AD2102F01E0DCD2202E209405
:140600003090A50132203092A501042FC1DF499108954A939F
:1406140044273CC088E991E0E42FFF27E80FF91F208022205F
:1406280021F4042F0F5FC5DF0AC088E991E0242E3324280ED9
:14063C00391EF10180818150808388E991E0E42FFF27E80F7A
:14065000F91F8081823031F4002706DF242F2F5F01EC6CDE82
:140664004B3049F4959896982090A60125BA969A95989698AE
:140678000AC0453041F4959896988FEF84BB2090A50125BAAD
:14068C00959A43954C3008F4C1CF499108954A935A93229751
:1406A00026E104E710E04CD1402F073008F437C02090A70156
:1406B40030907700321409F030C0409178005527413DE0E0C9
:1406C8005E0749F0423DE0E05E0781F0433DE0E05E0799F03D
:1406DC0017C08CE020907900821590F0822D813078F0082F88
:1406F00005DF0CC00027B8DE2091790002EC1EDE05C081E04F
:140704008093730001E0F8DE86E190E0998388832227332703
:1407180004E710E09DD12296599149910895A4DD62DD6CDD62
:14072C0078DDA8950AE810E0E9DD09C0A895AFDF2090A40196
:14074000222011F401E090DE64DFF6CF08952A923A920A9345
:140754008A939A93EA93FA932FB62A9284E68CBD22242DBCBA
:14076800002717C088E991E0E02FFF27E80FF91F2080222077
:14077C0069F083E08093A40188E991E0202E3324280E391EE1
:14079000F10180818150808303950C3038F32090A4012220F8
:1407A40021F0822D81508093A40129902FBEF991E991999124
:1407B800899109913990299018950A921A922A923A924A929E
:1407CC005A926A927A928A929A920A931A932A933A938A93EC
:1407E0009A93AA93BA93EA93FA930FB60A92AA92AA24A8959C
:1407F400ACB02A2D01E910E05DD0A99009900FBEF991E99194
:14080800B991A991999189913991299119910991999089900A
:14081C00799069905990499039902990199009901895A6D11C
:14083000AA24F80162816D5F87E0821768F442E007C0E42FE6
:14084400FF27E00FF11F2080A22443954617B8F30A2D01C03D
:14085800002797C170D1C22EB8014FEFAA24EE2487E08C15FD
:14086C0050F4FB01E281FF27E60FF71F43812C2D8B01D7DF45
:14088000A02EA41619F441E050E002C044275527042F4AC197
:140894002224F80121822082EF5FFE4F2082E150F140ED5FE1
:1408A800FE4F20823324309297012092960108956FD1C22E86
:1408BC00A8012FEF30E0FA01008111270F5F1F4FD5D05801C3
:1408D000FA01218033240215130549F0CF010296E081FF27CA
:1408E400E80FF91FC082FA01A0825BC131D15901A801FA0176
:1408F80020803180321491F0CF010296E181FF27E80FF91FD5
:14090C002080F5012082CA0101961FEFFC0100810F5FE5D08E
:14092000FC0100831CC14A935A93A801FA0121800081015085
:1409340002191FEFD8D0599149910895FED0C22EA80121975E
:1409480022242882AA2479C09E0101E910E0CCDF2090960139
:14095C0030909701222009F53320F9F4209092012092930126
:14097000288020929201809193018C3521F0822D853C09F0A6
:140984005EC02090960130909701C10101969093970180937B
:140998009601F101E40FF51F2090930120822C2C3324409056
:1409AC009601509097014214530458F4C2010196909397011A
:1409C00080939601F201E40FF51F288020822090940120923E
:1409D4009501288020929401809195018D3019F4822D8A30B0
:1409E80081F0FA016281772780919601909197010197E62F00
:1409FC00FF273396E817F907F1F46530E0F0A0909601B090A8
:140A10009701222420929201209293012092940120929501DA
:140A2400332430929701209296012A2D8A0114DFE02E0023BE
:140A380011F400270BC00A2D09C001E910E06FDFA02E80E05D
:140A4C00801708F47FCF0027219668C088819981803089074C
:140A600029F0E02FF12F21930197E9F708953A932A931A933A
:140A74000A9308956894DA92D12E04C0E894DA92D12ED32629
:140A880017FF04C0109500950F5F1F4F37FF04C030952095F6
:140A9C002F5F3F4F0BD0D7FE04C0109500950F5F1F4FD99037
:140AB0000895689401C0E894EA92FA928A93EE24FF2480E1A1
:140AC400000F111FEE1CFF1CE216F30618F0E21AF30A039530
:140AD8008A95A1F716F40E2D1F2D8991F990E990089568940D
:140AEC0001C0E8942A93FA92EA92FF24EE2420E1000FFF1C94
:140B0000EE1CE11610F0E11A03952A95B9F70EF40E2DE99028
:140B1400F99029910895A990B990C990D990E990F99008950A
:140B2800A990B990C990D990E990F9904991599169917991AB
:140B3C0008957A936A935A934A93FA92EA92DA92CA92BA9218
:140B5000AA9208955A934A93BA92AA920895A990B99049916D
:140B6400599108957A936A935A934A930895499159916991C7
:140B7800799108957A936A935A934A93BA92AA920895A99090
:140B8C00B990499159916991799108955A934A93DA92CA9215
:140BA000BA92AA920895A990B990C990D99049915991089577
:140BB400112319F0000F1A95FBCF0895112319F006951A9544
:040BC800FBCF0895C2
:00000001FF
